:020000002528B1
:080008008C00030E83018D0042
:100010000A088E008A0104088F000E281508810046
:100020000130180298009808031D1B281608980034
:100030000130190299000B110F0884000E088A0084
:100040000D0E83008C0E0C0E0900FF309200FF3065
:1000500093009313E4209315E52050201D089A0087
:100060001E089B001F089C003E3092201A0E0F397C
:10007000712092201A080F39712092201B0E0F391F
:10008000712092201B080F39712092201C0E0F390D
:10009000712092201C080F39712092202D284F28A2
:1000A000A001901C572820089C3C03195E287F2043
:1000B0002108A00090101019901451287F202108C9
:1000C0009D009010101990147F2021089E00901020
:1000D000101990147F2021089F009010101990147F
:1000E00008009E000A301E0203187A281E08303EBF
:1000F0007E287E280A301E02413E7E28080086198E
:100100007F28A720A9200830A200B6200310A10C48
:10011000A1138619A117A20B8528B62010118619E4
:100120001015B6289D00A920B620B6209417E0200F
:10013000B62008309E0094131D1C9417E020031075
:100140009D0CB6209E0B9B289413E020B6283230DD
:10015000D328D030AB28A2000130970001309600A0
:100160000E302202013C95000830BC289908031D7E
:10017000B628170899000800A3008B1FC1288B130D
:10018000BD28831601088312D03923078316640023
:10019000810083121508810016089800170899003D
:1001A0008B168B170800A200F430A300FC30A400CB
:1001B00022082307031C003424070318DC28080046
:1001C000E128140886000800E628E62813086600DF
:0201D000080025
:02400E00F93F78
:00000001FF
